:020000020000FC
:1000000056C937C20000000023C000004FC10000E5
:10001000000052C1000000000000000002030406BE
:10002000080C101820304060800002030406080C01
:10003000101820304080FF000406080C10182030F3
:10004000406080A0C00005050D050D0603030302F6
:100050004FB662FD20C070FF1CC165FDFCC057FE9D
:1000600001C00994C0919700C395C0939700C5E063
:10007000C519B8F3D0919700CD1B98F3C8E7089441
:1000800083FDC795C4BDC52DCC2321F4C0E083FDFD
:10009000C0E8C4BD09C171FF03C09598AC98C09871
:1000A000C52D089483FDC795C4BDC09399006B7F8F
:1000B000C52DCF3F09F443C0C0919800C395C093AC
:1000C000980070FF37C082FD05C09598AC98C09825
:1000D0004FBE18957860C091A000CC2391F0C091DC
:1000E0009800CA95D091A000CD1B58F0777FC091A1
:1000F0009800D0919F00CD1B08F41CC0209298005E
:1001000019C09598AC98C098C5E0CA95F1F7C09110
:100110007500CA95C2FD09C0C1FD05C095FFAB9829
:1001200095FD94980EC0AD980CC095FF949895FDE0
:10013000AB9807C09598AC98C0984FBE1895209280
:1001400099004FBE1895A5C0552021F095FF959AAE
:1001500095FDC09AAC989DC0552009F0AC9A95FFCA
:10016000C09895FD959895C0552021F095FFC09AAF
:1001700095FD959A95FF959895FDC0988AC095FF35
:10018000949A95FDAB9A95FFAB9A95FD949AC5E02C
:10019000CA95F1F7552021F095FF959A95FDC09AE3
:1001A000AC9877C095FF949A95FDAB9AAD9AC5E04F
:1001B000CA95F1F7552021F095FF959A95FDC09AC3
:1001C000AC9867C0AD9A95FF949A95FDAB9AC5E03F
:1001D000CA95F1F7552009F0AC9A95FFC09895FDA6
:1001E000959857C0AD9A95FFAB9A95FD949AC5E046
:1001F000CA95F1F7552009F0AC9A95FFC09895FD86
:10020000959847C095FFAB9A95FD949AAD9AC5E035
:10021000CA95F1F7552021F095FFC09A95FD959A62
:1002200095FF959895FDC09834C095FFAB9A95FDC4
:10023000949A95FF949A95FDAB9AC5E0CA95F1F70B
:10024000552021F095FFC09A95FD959A95FF9598B8
:1002500095FDC0981EC082FF1CC0C0917500C2FDF4
:100260000BC0C1FD11C095FF949A95FDAB9A95FF07
:10027000AB9A95FD949A0DC0C1FDF5CF95FF949A68
:1002800095FDAB9AAD9A05C0AD9A95FFAB9A95FDD9
:10029000949AC52DC095089483FDC795C4BDC0939D
:1002A00099002092970064604FBE18954FB6C0E148
:1002B000C8BF6E7F4FBE18953FB68F7EABB7A07498
:1002C000A2118061A0E0ABBFA9B7AE7FA9BF7894AF
:1002D000A0916600AA2349F0A92FAF7151F1A09116
:1002E0006600AA95A093660024C040E050E0A0B349
:1002F00096FDA095A2FD4FEF96FFA3E096FDA2E02C
:10030000A5BFAA27A064AABF8D7FA0B396FDA09524
:10031000A2FD5FEF451749F7A8E161FDA0936600D4
:10032000A92FAF7119F0A8E1A093660040938D004A
:100330008160A0916700AA2331F0A0916700AA957F
:10034000A093670007C0A92FAF7121F08061AA2791
:10035000A064AABF80FF48C0A0918D004A2F8E7F65
:10036000A92FAF71C1F0403F08F040EFA42FA29534
:10037000AF704A0F5091B000533069F0A695A69522
:1003800050FD01C0A69552FD03C0A41B4A2F03C017
:100390004A0F08F44FEFA09196004A1708F44A2F2D
:1003A0004093610071FF08C0A091610050919200DC
:1003B000A51710F050936100A09161004091630077
:1003C000A41B70F04091CF00A40B50F0A0916300EB
:1003D000A40FA093630040F4AFEFA093630004C0A8
:1003E000A0916100A093630040916300A0919200EE
:1003F0004A1708F04A2F542EA52DA03408F0686043
:10040000A0916000A395A093600051F0F894A9B763
:10041000A160A9BF84FF02C0A0E4ABBF3FBE189596
:1004200041E050916600552331F0A92FAF7119F4C6
:100430005A9550936600A0918D00A13018F020923B
:1004400090000DC02092910020929A00A0919000FF
:10045000AF5FA093900018F0AFEFA0939000F894D6
:10046000A9B7A160A9BF84FF02C0A0E4ABBF3FBE93
:1004700018953FB64CB55DB58F7EABB7A074A21191
:100480008061A0E0ABBFA9B7AE7FA9BF789481FD22
:1004900026C096FFA2E096FDA3E0A5BF8260A0B3B0
:1004A00096FDA095A2FF05C040936400509365009F
:1004B00033C196FFA3E096FDA2E0A5BFAA27A064E2
:1004C000AABF8D7FA92FAF7109F417C140E0A0B377
:1004D00096FDA095A2FD11C140938D0004C196FF29
:1004E000A3E096FDA2E0A5BF8D7F61FF6BC096FFE4
:1004F000A2E096FDA3E0A5BFAA27A064AABF8260E0
:100500004093880050938900A09086004A19B090CB
:1005100087005B09BB24A2E0EA2EA22C483CA0E0A5
:100520005A0730F4A0E1BA2EE22CAAE0AA2E27C086
:100530004836A1E05A0730F4A8E0BA2EE22CAFE02A
:10054000AA2E1DC0403DA2E05A0730F4A4E0BA2E06
:10055000E22CAEE1AA2E13C0403AA5E05A0730F4CF
:10056000A2E0BA2EE22CACE3AA2E09C04839A8E0DA
:100570005A0728F4A1E0BA2EE22CA8E7AA2EC42E2E
:10058000A0918A00CA1AD52EA0918B00DA0ADD202C
:100590002AF4AFEFC094D094CA1ADA0A20928C00E1
:1005A000CA14DE0418F4A1E0A0938C0040938A00E2
:1005B00050938B00409188005091890040938600B1
:1005C00050938700A09164004A1BA09165005A0BCC
:1005D00094FD7CC093FD7AC092FD76C056954795F8
:1005E00091FD72C05695479590FD6EC0D52EC42ED4
:1005F000D694C79461FD0CC0AC2DAC51AD2DA2407A
:1006000008F07BC0DD2021F4AC2DA85C08F475C097
:10061000A0E0EA2E97FD08C0E090C200A091B400CF
:10062000A33011F4E090CA00AAEFEA0EF22CF21CFB
:10063000CE18DF084FB74170A091B400A330A9F4E1
:10064000442329F095FD11C0F894906204C095FFF1
:100650000CC0F8949F7D9598AC98C098949AAD9AE8
:10066000AB9A71FD01C060687894442369F0A09151
:10067000B400A33031F4AFEFC094D094CA1ADA0AB0
:1006800003C040E050E022C0A091B400A33049F480
:10069000CC0CDD1CA5E0CA1AD20818F4A0E0CA2EC2
:1006A000D22CAFEFCA16D20418F04FEF50E00EC0B4
:1006B000F090A700CF9C412D000C441F50E008F0A3
:1006C00012C04FEF50E00FC05695479594FF07C0FA
:1006D000552309F04FEFA42FA6954A0F521D4F3F07
:1006E000520508F04FEF40938D00816061FF05C017
:1006F000AFE1A095A923AB299A2FA8E1A0936600AA
:10070000A92FAF7119F4AAE0A093660061FD04C09F
:10071000A92FAF7109F08F7EA6E0A0936700A92FE3
:10072000AF7119F4AAE0A0936700F894A9B7A1608B
:10073000A9BF84FF02C0A0E4ABBF3FBE189511E083
:100740000AC013E008C01AE006C01EE104C014E6A7
:1007500002C018EC00C005E1BB27BA95F1F70A9575
:10076000D9F71A95C1F708952AE338E709C020E3BD
:100770003CE806C02AE234EB03C025E238EC00C0B6
:10078000652CB1E05B2E12E095FD9F7D95FF906298
:10079000BB27AD9ABA95F1F7552009F0AC9ABA95F6
:1007A000F1F7AC98BA95F1F7AD98BA95F1F75520F5
:1007B00021F095FF959A95FDC09AB091A800BA9541
:1007C000F1F795FF959895FDC098B7E8BA95F1F7C0
:1007D0001A95D1F6022FB22FBA95F1F70A95D9F7EB
:1007E0003A9571F6AD9A562C0895221B39E0001FF8
:1007F0003A9509F40895221F211B18F4210F8894BB
:10080000F6CF0894F4CF622C722CB0E08894B395A4
:10081000221F331FE0F7379527958894912E802E5D
:10082000020B130B10F4192D082D10F4889401C03D
:100830000894661C771CBA9571F7172D062D08953C
:10084000322D11232AF43A9500951095031B130BB2
:10085000F894029F712C002D129F912C802C78947B
:10086000780C172D921C292DB4E06B2E2695179528
:1008700007956A94D9F7332321F000951095031B4F
:10088000130B0895089566FF21C01091740016950A
:10089000009173000795B0917700B01B0B2FB091BA
:1008A0007800B10B1B2F28F40038BFEF1B0740F076
:1008B00009C00F37120508F405C00FE710E002C0A9
:1008C00000E81FEF00937C0010937D00089566FF01
:1008D00039C000917C00B09179000B0F10917D0020
:1008E000B0917A001B1F20E030917D0033230AF481
:1008F0002A95B0917B002B1F1AF4203F40F00AC0CC
:100900002F3008F407C00FEF1FEF2FE003C000E007
:1009100010E020EF30916300B09192003B1718F483
:10092000332331F009C0B0917D00BB235AF004C0DD
:10093000B0917D00BB2332F40093790010937A00CC
:1009400020937B00089566FF2FC02091CD00009179
:100950007C00000F10917D00111F72DF11232AF41B
:100960000038BFEF1B0740F009C00F37120508F42D
:1009700005C00FE710E002C000E81FEF002352F0AF
:10098000B0916200B01B0B2F18F0013008F00AC0C4
:1009900001E008C000950F5FB09162000B0F08F0F6
:1009A00001C00FEF00937E00089566FF2DC02091D7
:1009B000CE0000917A0010917B0042DF11232AF4CF
:1009C0000130BFEF1B0740F009C00F3F120508F4CC
:1009D00005C00FEF10E002C001E01FEF112352F03D
:1009E000B0917E00B01B0B2F18F0013008F00AC048
:1009F00000E008C000950F5FB0917E000B0F08F07B
:100A000001C00FEF0093630008950FEF677FB72FCA
:100A1000B670E9F46860B0917400B83008F0677F90
:100A2000B0917400A1F00FEF10917400DEDEF89425
:100A3000B09170000B9F112D002D7894112309F0B7
:100A40000FEFB09195000B1710F4009195000093F3
:100A5000940008956BC001D374FFB2E074FDB1E05F
:100A6000B7B9B6B1B068B064B6B969DE74FFB2E0C8
:100A700074FDB1E0B7B9B6B1B068B064B6B9B6B19B
:100A8000B6FDFDCF04B115B1B6B1BF77B6B938D355
:100A900024E72093A30030E03093A400732E7694D3
:100AA000622E6694620E731E262D372D02171307D1
:100AB00078F08090A300B4E7B80DB093A3008090C5
:100AC000A400B0E0B81DB093A400260D371DEECFF2
:100AD0008090A3009090A4001091A400169500911E
:100AE000A300079516950795B091A300B00FB0939A
:100AF000A100B091A400B11FB093A20023E016950D
:100B000007952A95E1F72091AF002A9529F42092C4
:100B1000A3002092A4000AC02A9521F0800E911E05
:100B20002A95E1F78092A3009092A4000895209165
:100B3000AF00B6B1B6FDFBCF04B115B1B6B1BF770A
:100B4000B6B9B091A500B395B093A500B83060F1E7
:100B50002092A500B091CC00BB2321F1112329F0F4
:100B6000B091A600BF3F61F009C0B091A6000B177D
:100B700039F020F4BB2321F0BA9502C0B395E1F31C
:100B800000919200B093A600B83850F400ECBD3745
:100B900038F400E8B23720F400E4B73608F400E097
:100BA000009392007F7E0895B0919200B39511F06A
:100BB000B0939200B091A500B73009F47061089528
:100BC00002E3F894B091D0000B9F012D000C001FA0
:100BD0007894B09192000B1710F00091920000935E
:100BE000610000936300502E0093950008952092B9
:100BF0007300B8E0B09374000895209180003091A4
:100C00008100F8940CB51DB5200F311F3BBD2ABDE6
:100C10006160B0E1B8BF78942091710030917200AA
:100C20000093710010937200021B130B209173004C
:100C300030917400622E732EB4E08B2EB2E09B2EA6
:100C4000B0917400B43010F08A949A94B83010F0D7
:100C50008A949A94769467948A94E1F726193709CE
:100C6000992021F0169507959A94E1F7200F311FEE
:100C7000209373003093740008F00895BFEFB09391
:100C80007300B09374000895209182003091830026
:100C9000F8940CB51DB5020F131F1BBD0ABD616092
:100CA000B0E1B8BF7894089560FDFECFEDDF089500
:100CB000B091BE0000916E00023808F0B395003A82
:100CC00008F0B395B63008F0B5E09B2EBCE08B2E53
:100CD000B0917400B33030F48394839482FF02C0E7
:100CE00083948394B23030F48394839482FF02C05F
:100CF0008394839471FF03C0B3E09B2E822C1091E8
:100D000074000091730024E0169507952A95E1F789
:100D10000819120928F0B02FB250B12FB20910F4FF
:100D200002E010E0312F202F712E602E7694679410
:100D3000B92DB330E9F0B0FD05C0060D171D262D05
:100D4000372D06C0000F111F0250120922E030E0BB
:100D5000B92DB33068F02093840030938500009360
:100D60008000109381006092820070928300089549
:100D700000938400109385002093800030938100BD
:100D80006092820070928300089560FDFECF2091F2
:100D90008200220F30918300331FB72FB67021F0ED
:100DA0002091730030917400F8940CB51DB5020FBA
:100DB000131F1BBD0ABD6160B0E1B8BF78940895F0
:100DC00060612092760020E004C06061209276008D
:100DD00020E2B72FB67009F06F7E789460FD05C0F1
:100DE000B0917600BB2309F0089501E063FF0AC0CB
:100DF000B0917400B33008F002E0B0917400B630E6
:100E000008F003E071FF01C006E060FD06C0B0918C
:100E10007600BB2311F0789408951AE083FF1AE05E
:100E2000789400000000F89462FD03C014E183FF91
:100E300014E171FF01C018E7B4B530919900B31BFC
:100E4000B10B18F3B0917600B395B0937600B5E08E
:100E50003B2F6B2E722CB8B1B072B21709F073949D
:100E60003A95C9F77394761488F464FFB2CF6F7E15
:100E70003CB56DB47090730080907400370D681CA1
:100E80006BBC3ABD6160B0E1B8BFA3CF64FDA1CF38
:100E90000A9509F0BACF7894089571FF0AC0B0910D
:100EA0006D00B395B0936D0060FD0CC020926D0095
:100EB00009C060FD07C064FD05C067FD03C0BF91A8
:100EC000BF918AC408952091840030918500F894E0
:100ED0000CB51DB5020F131F1BBD0ABD6160B0E14B
:100EE000B8BF78940895EFDF00E063FF03C064FFAC
:100EF00001C001E0F89410916E00B7E01B9F212D16
:100F0000102D7894200F26951795269517952695E0
:100F1000179510936E00183718F4B8E7B0936E0069
:100F200000916E00B0916F000B1720F060629598F1
:100F3000AC98C09860FDFECF0895F894949AAD9A4D
:100F4000AB9A82FF07C0E2E0F1E073FF03C0B5E0B7
:100F5000BA95F1F7B0917400BC7F81F0552021F073
:100F600095FF959A95FDC09AB6E0BA95F1F795FF71
:100F7000959895FDC098B5E0BA95F1F795FF9498CE
:100F800095FDAB98B2E0B0937500ABC0F89495FFB7
:100F9000C09895FD959882FF0DC0E2EFF0E073FFD9
:100FA0000BC0AD9A95FFAB9A95FD949AB5E0BA95B2
:100FB000F1F702C0ECEAF0E062FF03C0552009F04F
:100FC000AC9AB3E0B09375008CC0F894949AAD9A43
:100FD000AB9A82FF07C0E2EEF0E073FF03C0B5E01A
:100FE000BA95F1F7B0917400BC7F81F0552021F0E3
:100FF00095FFC09A95FD959AB6E0BA95F1F795FFE1
:10100000C09895FD9598B5E0BA95F1F795FFAB9826
:1010100095FD9498B4E0B093750063C0F894AC98D3
:1010200082FF0DC0E2EDF0E073FF0BC095FF949AD4
:1010300095FDAB9AAD9AB5E0BA95F1F702C0E4EA36
:10104000F0E062FF06C0552021F095FF959A95FDCE
:10105000C09AB5E0B093750044C0F894949AAD9AE4
:10106000AB9A82FF07C0EFEBF0E073FF03C0B5E07F
:10107000BA95F1F7B0917400BC7F51F0552009F09A
:10108000AC9AB6E0BA95F1F7AC98B5E0BA95F1F73D
:10109000AD98B6E0B093750024C0F89495FF95988C
:1010A00095FDC09882FF10C0E5E1F1E073FF0EC02E
:1010B00095FF949A95FDAB9A95FFAB9A95FD949AFE
:1010C000B5E0BA95F1F702C0E4EBF0E062FF06C0CC
:1010D000552021F095FFC09A95FD959AB1E0B09307
:1010E000750067FF0AC00CD0B5E0BA95F1F7B5E01E
:1010F000BA95F1F79498AD98AB986F7D7894089570
:1011000023EA30E0F9019598AC98C098949AAD9A8A
:10111000AB9A6B7F0895ACEAB0E00FEF0D930D939F
:101120000D930D9303E00D9304E00D930BE00D93ED
:1011300003E00D9301E00D9301E00D93A8EBB0E007
:1011400001E00D930FEF0D930D930FEF0D930D93A2
:101150000D9303E00D9306E00D930FEF0D930D93A8
:1011600005E20D9300ED0D930AEF0D930AEF0D9339
:1011700004E00D930DE00D9301E00D9300E00D935D
:101180000AE70D930FEF0D9301E00D930895209161
:10119000BF0009E011E0223011F405E011E0233036
:1011A00011F405E012E0243011F405E013E02530DD
:1011B00011F409E017E0263011F400E010E000938C
:1011C0009F001093A0002091B3008B7F233009F47F
:1011D0008460777F233009F47860B091B400B33035
:1011E00019F09F7DB1FD90629F7BB091B500B1FD7C
:1011F0009064B22FB23011F0886001C0877F0895EB
:10120000ECE1F0E00091AC000A95E00FF21DB49122
:10121000B093CD000091AD000A95E00FF21DB4919E
:10122000B093CE006DDF0895EAE2F0E00091C700D0
:101230000A95E00FF21DB491B093CF0061DF0895DD
:10124000E8E3F0E00091B2000A95E00FF21DB491DE
:10125000B093D00055DF08950895B091C8000FEF06
:101260001CE0B23011F400EA1AE0B33011F402E8E5
:1012700015E000936F001093700008950895209179
:10128000C2003091C30097FF02C020E03FEFB32FB0
:10129000B21B6B2EB25810F4B2E86B2E00E003952F
:1012A000609EB12DB058D8F30093A7000895F8942C
:1012B000E3E0F0E0B9E0B7BFB491B078C1F3F894DF
:1012C000A895B1B5B861B1BDB0E0B1BDB4E0BEBFE5
:1012D000BFE5BDBF15DFB0E0B8BBB1E1B7BBB8E259
:1012E000B5BBB8E3B4BBB0E1B2BBB0E3B1BB222441
:1012F000A0E0B0E02D92AA31E9F7A0E6B0E00FEF50
:101300002D920A95E9F707DF87D241DF79DF8CDF7D
:1013100097DFA2DFA2DFB2DFB2DF0091C40000934B
:10132000A800EEDEB2E0B3BFB2E0BEBDB2E0B5BD34
:10133000F8940FDA19DA09DA1ADA07DA1BDA05DAB9
:10134000F6D207DA06DA03DAB1E5B8BFB9BFB0B74B
:10135000B860B0BFB6B1B460B6B9F1D978947ADBF1
:10136000B0E4BBBFBB27B064BABF8D7FF2D9B1E098
:10137000B0936900626025E0B0918C00BB2309F452
:1013800025E0DFD9B0918D00B230A8F3B92FBF713D
:1013900000918F0000938E00B0938F00B01759F723
:1013A0002A9551F76D7F96FFB3E096FDB2E0B5BF89
:1013B000BB27B064BABF8D7FCAD9C3D902E0B92FA9
:1013C000BF7109F400E0B0918D00B017B0F3F8944C
:1013D000CBD9CAD9C9D97894BCD920927F00B09111
:1013E000B400B33009F472C0ACD9B091B800B130D8
:1013F00008F46CC0B0916900B13008F467C0B92F2F
:10140000BF71C1F0B0918D00BF3F08F45FC0F89488
:10141000B4D978949CD9B0918D00B130C0F7F894CC
:10142000A3D991D9A1D9789492D9B0918D00BF3F19
:10143000B0F3AFC2B8E09B2E9068F89420DF7894A8
:1014400086D9F8949F771BDF80908D00B0918D0036
:10145000BF37789408F442C072D9F8948ED9789442
:101460009A9451F7B82DB550B093C30072D9F8943F
:1014700000D262D27894BAE09B2E9068F894FFDE96
:10148000789465D9F8949F77FADE80908D00B091BA
:101490008D00BF37789478F752D9F89465D953D92D
:1014A00063D978949A9449F7B82DBB5FB093C20082
:1014B00050D9F894DED14FD2789449D9F894DFDE30
:1014C0007894B0918D00BF3FC0F363C200918D004E
:1014D000B0917F000B1710F000937F0038D901E026
:1014E000B091B400B35009F405E0B0918D00B0178D
:1014F00008F075CFF89441D940D93FD9789429D9CB
:101500002092690020926A0020926B00B0916A00DC
:10151000B395B0936A00BF3F69F5B0916B00B39586
:10152000B0936B00B091C60009E1BA9559F002E39F
:10153000BA9541F00DE7BA9529F00AEFBA9511F086
:1015400020926B00B0916B00B017A0F0B0916B00CF
:10155000BA95B0936B00B4EBB0936A00B091C5003C
:10156000B093A800F89409D97894B091C400B093CE
:10157000A800EDD8E8D8B0916600BB2321F4B92FBC
:10158000BF7109F4F7CEB0918D00B63008F4BECF2C
:10159000B091B400B35009F0DAD8B0916600BB2323
:1015A00009F4E8CEF894ACDD20926100209262004C
:1015B00020926300522C7894B091B100B0939600C1
:1015C00020927700209278002092790020927A0071
:1015D00020927B002092A50060E070E020926E00D7
:1015E00006DBB8E0B093A5007061A9D874FFB2E043
:1015F00074FDB1E0B7B9B6B1B068B064B6B9B6B110
:10160000B6FDFDCF04B115B1B6B1BF77B6B91123A0
:1016100009F00FEF0093A6008ADAB8E0B093A500B6
:1016200070618090B300B2E0B093B300B0DD8092FF
:10163000B300F894BFEFB0939200C2DAB0916100AA
:10164000B0939200B0939300B09394007894B1E07B
:10165000B0936100B09363005B2EB0939B00B09198
:101660009100B0939A007160726020926D00F5DC79
:1016700014DDC3DABCDA1CDB04C089DD2092A500CE
:101680007F7E95FFB6E095FDB0E0B7B99EDB05DC47
:101690001ADCF8D828DC51DCB0DA06DB09DB75DBB4
:1016A000B7E0B7B98DDBF9DB0EDCEDD8AED91BDCCA
:1016B0006DDCA3DAF9DAFCDA68DB95FFB0E095FDC2
:1016C000B6E0B7B982DBE9DBFEDB01D90CDC7DDCFF
:1016D00094DAEADAEDDA59DB95FFB6E095FDB0E091
:1016E000B7B96EDBDADBEFDB2ED9FDDB97DC85DA11
:1016F000DBDADEDA4ADBB7E0B7B967DBCEDBE3DBA8
:1017000054D9F1DBAADC79DACFDAD2DA3EDB95FF05
:10171000B0E095FDB6E0B7B953DB74FFB2E074FDFD
:10172000B1E0B7B9B6B1B068B064B6B9B6DBCBDB7F
:10173000DADBB3DC62DAB8DABBDAF9D926DB71FFBF
:1017400025C067FD23C0B0919500B0939200B0937F
:101750009300B0919100B0939A00B1E0B0939B00D8
:1017600014E624E1B0916D00B11750F07D7F7460F4
:1017700020936C00BFEFB0939200B093930006C02B
:10178000B0918D00B13008F07CCF26C072FF10C040
:1017900067FD0EC0B0916C00BA9511F47B7F6DCFE0
:1017A000B0936C00B0918D00B13008F06ACF14C0D6
:1017B000B0919000B23880F4B92FBF7121F4B0918C
:1017C0006600BB2349F0B091740000EF67FF01C0D1
:1017D00000E6B01708F455CFF89492DC8090B3007F
:1017E000B2E0B093B300D3DC8092B30020926100EA
:1017F0002092620020926300522C209296007E7FFD
:1018000078949DD77DDCB92FBF7129F4B091660023
:10181000BB2309F4AFCD76CEEDE0F0E023D00A355E
:1018200009F01BC0EEE0F0E01DD0053A09F015C04C
:101830003AE0ACEAB0E0E3E0F0E014D00D9331968A
:101840003A95D9F735E1A8EBB0E0EFE0F0E00AD047
:101850000D9331963A95D9F702C05DDC0AD0E4E2E7
:10186000F0E00895E199FECFEEBBFFBBE09A0DB327
:1018700008951ED03AE0ACEAB0E0E3E0F0E00D916C
:101880000FD031963A95D9F735E1A8EBB0E0EFE00B
:10189000F0E00D9105D031963A95D9F712D0089520
:1018A000E199FECF0DBBEEBBFFBBE29AE19A089532
:1018B000EDE0F0E00FEFF4DFEEE0F0E00FEFF0DF4F
:1018C0000895EDE0F0E00AE5EBDFEEE0F0E005EA98
:1018D000E7DF08953091A9000091AA00313011F49A
:1018E0000093B000323011F40093B100333011F4A2
:1018F0000093B200343011F40093BE00353011F47F
:101900000093C700363011F40093BF00373011F454
:101910000093B300383011F40093C800393011F44B
:101920000093B4003A3011F40093B500089525E017
:1019300010D72A95E9F7089517D719D71BD71DD7C0
:1019400002D712D714D716D718D7FDD60DD70FD771
:1019500011D713D7089511D70DD709D705D7F3D6C7
:101960000CD708D704D700D7EED607D703D7FFD6B2
:10197000FBD608958090A9009090AA00F5D6F4D6E1
:10198000F3D6E1D68A94D1F7F8D6DDD69A94E1F76A
:101990000895F894D1DF7894CADFC9DFB1E0B0933D
:1019A000A900B1E0B093AA002092AB00F894E2DF66
:1019B0007894B5E06B2E70908D00CBD6B0918D00F1
:1019C0007B16C9F7B13018F0BF3F40F107C082DF86
:1019D000F8944FDFB1DFB8E0B1BDA9DF6A9459F7E1
:1019E000B091AB00B395B093AB00B33008F4DECF49
:1019F0009EDFB091AA00B395B093AA00F894B0917D
:101A0000A900BA95E6E4F0E0EB0FF21D049178949A
:101A10000395B091AA00B01708F4C6CF88DF87DF1E
:101A2000B091A900B395B093A900B091A900BB30C3
:101A300008F4B7CF70DBF8941CDFB8E0B1BD77DFF6
:00000001FF
